:020000040000FA
:04000000C5EF00F058
:0800080000D09EAA1000F29E38
:100010009E9AAE50806F410E805DD8B43CEF00F0E8
:10002000460E805DD8B442EF00F0570E805DD8B424
:1000300048EF00F05A0E805DD8B44EEF00F0510E3C
:10004000805DD8B438EF00F0490E805DD8B454EF2D
:1000500000F0F28CF28E805132EC00F00D0E32EC9A
:1000600000F011009E98AD6EACA234EF00F01200CB
:100070008292829429EF00F083808382828282843C
:1000800029EF00F0839083928282828429EF00F02E
:10009000828282848380839229EF00F0828282842C
:1000A0008390838229EF00F0FF0E936E80CF81F062
:1000B00081CF82F082CF83F083CF84F0090E32ECBF
:1000C00000F0A4EC00F09FEC00F09AEC00F095EC4E
:1000D00000F090EC00F08BEC00F086EC00F081EC8E
:1000E00000F0200E32EC00F0A9EC00F0AEEC00F0D5
:1000F000B3EC00F0B8EC00F0090E32EC00F029EFA0
:1001000000F082AFC1EF00F0BDEF00F082ADC1EFB3
:1001100000F0BDEF00F082ABC1EF00F0BDEF00F0EA
:1001200082A9C1EF00F0BDEF00F082A7C1EF00F09F
:10013000BDEF00F082A5C1EF00F0BDEF00F082A39B
:10014000C1EF00F0BDEF00F082A1C1EF00F0BDEF04
:1001500000F084ADC1EF00F0BDEF00F084AFC1EF5F
:1001600000F0BDEF00F081A9C1EF00F0BDEF00F09D
:1001700083A1C1EF00F0BDEF00F0300E32EC00F0D3
:100180001200310E32EC00F01200846AFF0E926E03
:10019000FF0E936E990E946EC00E956E966A240EA5
:1001A000AC6E400EAF6E9D8A900EAB6EF28CF28EEE
:0401B000D8EF00F094
:020000040030CA
:0E000000FFFAFDFEFFFEFAFFFFFFFFFFFFFF0E
:00000001FF
